:100000000C94CD020C94EA020C94EA020C94EA02DD
:100010000C94EA020C94EA020C94EA020C94EA02B0
:100020000C94EA020C94EA020C94EE250C94C0267F
:100030000C94E0200C94EA020C94EA020C94EA027C
:100040000C94EA020C94EA020C94EA020C94EA0280
:100050000C94EA020C9468210C94EA020C94EA02D3
:100060000C94EA020C94EA020C94EA020C94EA0260
:100070000C94EA020C94EA020C94EA020C94EA0250
:100080000C94EA020C94EA020C94EA020C94EA0240
:100090000C94EA020C94EA020C94EA020C94EA0230
:1000A0000C94EA020C94EA020C94EA02AE05AE0546
:1000B000DA05DA0542066006780778076B0604075A
:1000C000150715072D2754274C2854274C28A027FF
:1000D000C3274C281A2829285F00600061001400FB
:1000E0001A000800150017001C0018000C00120070
:1000F00013005C005D005E000400160007000900AC
:100100000A000B000D000E000F00280059005A00D5
:100110005B001D611B640641194200002C62000057
:1001200005781174107149004A004B002900A8009D
:10013000AA00A900AE004A004E004B004D0000008E
:100140004C0052004E002B00000000000000000098
:100150005000510052004F002A00500051004F0043
:10016000E000E2000100035100002C620000E70003
:10017000E600E4005300000000001E001F00200005
:100180002100220023002400250026002700000073
:1001900000000000350000002D002E0031002F006F
:1001A0003000330034002A00000000000000E000AE
:1001B000E2000351010000002C620000360037000D
:1001C00038000000000000003A003B003C003D0009
:1001D0003E003F004000410042004300000000009C
:1001E0000000440045000000000000000000000086
:1001F000000000004C00000000000000E000E200F1
:100200000100010000002C620000E700E600E400AD
:1002100000047F3F1F643214643214783C1E1E14A5
:100220000A052223252628292A2C2D2F3032333562
:1002300036383A3B3D3E4042434547494A4C4E5092
:1002400051535557595A5C5E6062646668696B6DBC
:100250006F71737577797B7D7F81838587898A8CC0
:100260008E90929496989A9C9E9FA1A3A5A7A8AAC7
:10027000ACAEAFB1B3B4B6B8B9BBBCBEBFC1C2C3FC
:10028000C5C6C7C9CACBCCCDCED0D1D2D2D3D4D596
:10029000D6D7D7D8D9D9DADADBDBDBDCDCDCDCDCBF
:1002A000DDDDDDDDDCDCDCDCDCDBDBDBDADAD9D997
:1002B000D8D7D7D6D5D4D3D2D2D1D0CECDCCCBCA25
:1002C000C9C7C6C5C3C2C1BFBEBCBBB9B8B6B4B34B
:1002D000B1AFAEACAAA8A7A5A3A19F9E9C9A9896E1
:1002E0009492908E8C8A89878583817F7D7B7977B4
:1002F0007573716F6D6B6968666462605E5C5A5994
:1003000057555351504E4C4A4947454342403E3D54
:100310003B3A3836353332302F2D2C2A29282625E2
:100320002322FFAA7F5540000101010101010101C3
:100330000102020202020202020203030303030398
:100340000303040404040404040505050505060666
:100350000606060707070707080808080909090924
:100360000A0A0A0B0B0B0C0C0C0D0D0D0E0E0E0FCA
:100370000F0F10101111111212131314141515165A
:10038000161717181819191A1A1B1B1C1D1D1E1ECB
:100390001F2020212222232424252626272829291C
:1003A0002A2B2C2D2D2E2F30313232333435363747
:1003B00038393A3B3C3D3E3F404142434445464745
:1003C00048494A4C4D4E4F50515354555658595A1E
:1003D0005B5D5E5F616264656668696B6C6D6F70C2
:1003E00072737577787A7B7D7E8082838587888A31
:1003F0008C8E8F91939596989A9C9EA0A2A3A5A768
:10040000A9ABADAFB1B3B5B7BABCBEC0C2C4C6C963
:10041000CBCDCFD1D4D6D8DBDDDFE2E4E7E9EBEE1C
:10042000F0F3F5F8FAFDFF0E0341006C0070006870
:10043000006100390000001A0357006F0072006C61
:1004400000640073007000610077006E00300030BF
:100450000000000403090409023B00020100A0FAA5
:10046000090400000103010100092111010001221A
:100470004000070581030800010904010001030091
:10048000000009211101000122B6000705820320A6
:100490000001120100020000000853572A69010000
:1004A0000102000105010902A10185020901A10063
:1004B0000509190129081500250195087501810212
:1004C0000501093009311581257F950275088106DE
:1004D00009381581257F950175088106050C0A38B4
:1004E000021581257F950175088106C0C0050109A7
:1004F00080A101850319012AB700150126B70095CF
:100500000175108100C0050C0901A10185041901C4
:100510002AA002150126A002950175108100C005D0
:10052000010906A1018506050719E029E71500253F
:10053000019508750181020507190029EF150025AD
:100540000195F075018102050819012905950575C8
:10055000019102950175039101C005010906A101F0
:10056000050719E029E715002501950875018102A5
:100570009501750881010507190029FF150026FF5F
:10058000009506750881000508190129059505756E
:10059000019102950175039101C011241FBECFEF97
:1005A000DAE0DEBFCDBF11E0A0E0B1E0EEEFF2E5B2
:1005B00002C005900D92A43CB107D9F722E0A4EC4B
:1005C000B1E001C01D92A43FB207E1F70E947D1384
:1005D0000C947D290C94000081E0089581E0089539
:1005E0000C94EE0208950C94F2021F93CF93DF93C4
:1005F00000D000D01F92CDB7DEB749835A836B83FA
:100600003091C70189819A81311114C0662359F054
:10061000222349F00E94B509182F682F89819A81F9
:100620000E945E0903C00E948909182F69817A819E
:10063000812F04C00E94B50969817A810F900F90C3
:100640000F900F900F90DF91CF911F910C94EF10AE
:10065000FC01262F408151816281738184810C9439
:10066000F50281E00895CF93DF93EC0160E00E94F2
:100670002803BE01DF91CF910C94F3020C94351244
:100680000C94311208950E9408080E9442032FEF33
:1006900084E39CE0215080409040E1F700C00000DE
:1006A0000C948E210F931F93CF93DF938C0161E005
:1006B0000E942803EC01B8010E94F002882309F48B
:1006C00044C0B801CE010E942B1F8823F1F1B8016C
:1006D000CE010E943F1D8823C1F1B801CE010E94C6
:1006E000871E882391F1B801CE010E94451C882302
:1006F00061F1F8018281882309F1CB358DE5D807B6
:10070000C1F050F4C115FCE5DF0781F0CF3DDC45B9
:10071000A9F40E94EC0E19C0CC35EDE5DE0761F0BE
:10072000CD35DD4559F40E942F0E08C00E944303C9
:100730000CC00E94380E02C00E943B0EC801DF911F
:10074000CF911F910F910C94EC0280E0DF91CF913B
:100750001F910F9108950E94C2200C94D1030E9412
:10076000D4030C94C82008950C94B30381E0089539
:10077000CF93C82F0E94B603882329F0C1FD02C081
:100780005B9A01C05B98CF910895539A5B9A089544
:10079000CF93C82F0E94B4038C2F0E94B803CF912F
:1007A000089580E00C94C8030E94871F0C94C8032E
:1007B0000E94871F9091C601891721F08093C6017E
:1007C0000C94C8030895CF93DF93CDB7DEB72B9772
:1007D0000FB6F894DEBF0FBECDBF4F835887698731
:1007E0007A878B8761110E947B0D9E012F5F3F4F9F
:1007F00086E0F90111928A95E9F785E0FE013796C6
:10080000D90101900D928A95E1F789819A814C81F5
:100810005D81452B31F09F3F31F491E08F3F19F41A
:1008200003C091E001C090E090FF09C049815A8166
:100830006B817C818D819E810E949C0C05C0C901C9
:100840000E9431038111F2CF2B960FB6F894DEBFD0
:100850000FBECDBFDF91CF910895FC0180819181C2
:100860000E94F7090895CF93882309F4A4C0C82FE4
:100870008238C1F40E94871F81FD9DC069E3809189
:100880000201909103010E947D200E949D0D2FEF97
:1008900081EE94E0215080409040E1F700C00000DC
:1008A00069E319C0833801F50E94871F80FD83C06A
:1008B00063E580910201909103010E947D200E94D6
:1008C0009D0D2FEF81EE94E0215080409040E1F7A4
:1008D00000C0000063E580910201909103010E9435
:1008E0008820CF910C949D0D8438C1F40E94871FFD
:1008F00082FD61C067E480910201909103010E9432
:100900007D200E949D0D2FEF81EE94E021508040CC
:100910009040E1F700C0000067E4DDCF8CEF8C0F62
:10092000813AD0F46C2F80910201909103010E94D2
:10093000FD1F882349F06C2F8091020190910301E3
:100940000E9488200E949D0D6C2F80910201909141
:1009500003010E947D20C5CF80E28C0F883048F4CF
:10096000C77081E001C0880FCA95EAF70E945E0D4A
:10097000B8CFEBE5EC0FE33040F4F0E0E65AFE4F81
:10098000808190E0CF910C94BB1FE8E5EC0FE7313C
:1009900050F4F0E0EE0FFF1FE45DFE4F8081918187
:1009A000CF910C94D11FCD3E30F08C2F0E940214B9
:1009B000CF910C94D414CF910895882309F464C086
:1009C000823879F40E94871F81FF5EC069E38091BD
:1009D0000201909103010E947D200E949D0D69E318
:1009E00010C08338B1F40E94871F80FF4DC063E5BB
:1009F00080910201909103010E947D200E949D0D33
:100A000063E580910201909103010E9488200C947B
:100A10009D0D843879F40E94871F82FF35C067E4FA
:100A200080910201909103010E947D200E949D0D02
:100A300067E4E7CF9CEF980F913A10F4682FE1CF6D
:100A400090E2980F983050F4877091E001C0990FB0
:100A50008A95EAF7892F0E94640DD9CF9BE5980FFC
:100A6000933020F480E090E00C94BB1F98E5980F41
:100A7000973120F480E090E00C94D11F8D3E20F05F
:100A80000E945D140C94D41408951F93CF93DF93A8
:100A9000182FEB010E943304209741F08FE99FE06B
:100AA0000197F1F700C000002197F6CF812FDF9169
:100AB000CF911F910C94DD04893319F060E070E050
:100AC00002C060E570E00C944505882321F00E9487
:100AD0005E0D0C949D0D0895882321F00E94640DF5
:100AE0000C949D0D0895CF92DF92EF92FF920F9399
:100AF0001F93CF93DF937C01D62FC72FFC01128168
:100B0000058102950F700E94540D8823B9F01123BE
:100B1000A9F08C2F807F803421F080E28D0F883007
:100B200068F08091C20282FD09C082E00E94FD0D42
:100B30000E94540D91E0D82ED92601C0D12CCC2E84
:100B4000C2948FE0C8228C2D90E08C30910508F083
:100B5000CFC1FC01EA5AFF4F0C94D8288C2F807F1C
:100B6000CF70882311F0C295C07F112399F0CC2358
:100B700009F4AAC180E28D0F883010F0D11104C0B1
:100B80008C2F0E945E0D03C08C2F0E946E0D0E9460
:100B90009D0D9AC18D2F0E94DD04CC2309F4A8C1BC
:100BA00080E28D0F883038F1DD2329F18C2F0E94EF
:100BB000740D24C08C2F807FCF70803211F0C295CD
:100BC000C07FDD2319F0D130A1F13DC08091C20278
:100BD00082FF17C0112349F0CC2329F08C2F0E94EB
:100BE0005E0D0E949D0D80E070C180E00E94DD04DA
:100BF000CC2309F47DC18C2F0E94640D0E949D0DB1
:100C000077C1112371F0002341F0013031F40E94CB
:100C10007E0D8C2B0E94860D6BC10E947E0D8C2B4D
:100C20001DC0002319F0013009F462C10E94930D28
:100C300025C0112321F0063008F05AC10EC005303E
:100C400008F056C11BC0112361F0002331F0F701F9
:100C5000858180FF39C18F7085838C2F0E94650547
:100C600047C1002359F0D93309F03FC1FFEF07EE28
:100C700013E0F15000401040E1F735C18C2F0E9485
:100C80006C0536C18C2F86958695837019F081305E
:100C900061F02EC1112321F08D2F9C2F937002C083
:100CA00080E090E00E94BB1F2BC1112321F08D2F0B
:100CB0009C2F937002C080E090E00E94D11F20C161
:100CC0008D2F112319F00E94021402C00E945D149E
:100CD0000E94D41415C18C2F837009F047C01111E4
:100CE0000BC12D2F229526952770220F220F6D2FD5
:100CF0006F70862F90E0A0E0B0E0022E04C0880F55
:100D0000991FAA1FBB1F0A94D2F7D4FF10C04FE04F
:100D100050E060E070E004C0440F551F661F771F6D
:100D20002A95D2F7409550956095709503C040E0A4
:100D300050E0BA01C695C695C3708A019B01082B85
:100D4000192B2A2B3B2BC901B801C23049F058F4AA
:100D5000C13019F00E947408CFC00E946208CCC054
:100D60000E948608C9C00E946008C6C0112319F0FD
:100D70008C2F817001C08695882309F4BDC02D2F6A
:100D8000229526952770220F220F6D2F6F70862FC8
:100D900090E0A0E0B0E0022E04C0880F991FAA1FC7
:100DA000BB1F0A94D2F7D4FF10C04FE050E060E0C0
:100DB00070E004C0440F551F661F771F2A95D2F7B5
:100DC000409550956095709503C040E050E0BA01A1
:100DD000C695C695C3708A019B01082B192B2A2B37
:100DE0003B2BC901B801C23049F058F4C13019F0A9
:100DF0000E94390981C00E9427097EC00E944B09C8
:100E00007BC00E949A0878C0CF70112339F08C2FD4
:100E10000E94C0088D2F0E9465056EC08D2F0E9414
:100E20006C058C2F0E94E10867C0D23F21F128F4A5
:100E3000D03F41F0D13FC1F043C0D33F19F1D43F7F
:100E400079F03EC0112341F0053008F051C08C2FDD
:100E50008F710E9406094CC0063008F049C0F7CFD8
:100E60008091C20282FF18C0112339F08C2F8F713C
:100E70000E94C0083DC01123C9F38C2F8F710E94BE
:100E8000E10836C0112329F08C2F8F710E94AB0826
:100E90002FC00E94A6082CC0112349F0CF718C2FBF
:100EA0000E94C00863E08C2F0E94E20D21C081E007
:100EB0000E94FD0D0230E0F082E00E94FD0D18C09E
:100EC000112331F0002391F28D2F0E94330410C0C2
:100ED000002399F2D93349F41FEF27EE33E0115084
:100EE00020403040E1F700C000008D2F0E94DD045B
:100EF00088EF8C0D843020F40E94871F0E94C80365
:100F0000DD20C9F00E94500D80FD15C0F70112824E
:100F10000E944A0D0E94C008C7010E94BC070E949F
:100F20004A0DDF91CF911F910F91FF90EF90DF90CD
:100F3000CF900C94E108DF91CF911F910F91FF901A
:100F4000EF90DF90CF9008950F931F93CF93DF938F
:100F5000EC01688179818A810E94020A8C010E94D9
:100F60005D090E944E08B801CE010E947305DF9111
:100F7000CF911F910F910895CF93DF93EC0198814A
:100F800089812B813C81232B31F08F3F31F481E02B
:100F90009F3F19F403C081E001C080E080FD1DC0C7
:100FA000CE010E945203811110C00E94540D88236B
:100FB000A1F08A81882389F08091C20282FD0DC050
:100FC00082E0DF91CF910C94FD0DCE010E94A40729
:100FD000CE01DF91CF910C943303DF91CF9108952F
:100FE00080E090E00E94BB1F80E090E00E94D11F53
:100FF0000E947B0D0E949D0D0E9405160C94D41436
:1010000080910201909103010E9493200C94F007BB
:101010000E946B0D0C94000892959F70963079F0A9
:1010200010F4925001C09A50923068F4803F69F0F9
:1010300018F4883E40F409C0843F29F406C0883E75
:1010400020F0813F11F080E0089581E00895FC01D7
:10105000808191810E94F7090E940C080895CF9326
:10106000DF9300D000D01F92CDB7DEB70F900F9066
:101070000F900F900F90DF91CF910895CF93DF9352
:1010800000D000D000D0CDB7DEB726960FB6F894CA
:10109000DEBF0FBECDBFDF91CF91089508950895B3
:1010A0000C944F080C9450080E9452086093E5017C
:1010B0007093E6018093E7019093E8010C94F007A8
:1010C0000C9454080F931F930091E5011091E601D1
:1010D0002091E7013091E801602B712B822B932B3B
:1010E0001F910F910C9454080F931F930091E501E9
:1010F0001091E6012091E7013091E801602371230E
:10110000822393231F910F910C9454080F931F93E4
:101110000091E5011091E6012091E7013091E8018D
:1011200060277127822793271F910F910C945408F1
:101130000C944F080E9498086093E1017093E201BB
:101140008093E3019093E4010C94F00760E070E079
:10115000CB010C949A080F931F9341E050E060E09C
:1011600070E08A019B0104C0000F111F221F331F72
:101170008A95D2F7C901B8011F910F910C949A0872
:101180000F931F9341E050E060E070E004C0440F13
:10119000551F661F771F8A95D2F78091E1019091C4
:1011A000E201A091E301B091E4018A019B01082BC7
:1011B000192B2A2B3B2BC901B8011F910F910C94BD
:1011C0009A080F931F9341E050E060E070E004C084
:1011D000440F551F661F771F8A95D2F7409550958B
:1011E000609570958091E1019091E201A091E301F9
:1011F000B091E4018A019B01082319232A233B2390
:10120000C901B8011F910F910C949A080F931F9375
:1012100041E050E060E070E004C0440F551F661FDD
:10122000771F8A95D2F78091E1019091E201A09118
:10123000E301B091E4018A019B01082719272A27BD
:101240003B27C901B8011F910F910C949A080F9385
:101250001F930091E1011091E2012091E30130918F
:10126000E401602B712B822B932B1F910F910C9417
:101270009A080F931F930091E1011091E2012091D0
:10128000E3013091E40160237123822393231F91B2
:101290000F910C949A080F931F930091E101109104
:1012A000E2012091E3013091E40160277127822758
:1012B00093271F910F910C949A0808952DE0929F07
:1012C000800D1124E82FE695E695E695877051E0AC
:1012D00001C0550F8A95EAF785E0E89FF0011124D7
:1012E000E853FE4F20E030E070E04081CB01022E59
:1012F00002C0969587950A94E2F7817081958427BC
:101300008523842781932F5F3F4F2530310569F76F
:1013100008952DE0929F800D1124682F66956695A3
:101320006695982F977085E0689FB001112440E082
:1013300050E080E0FB01E40FF51FE853FE4F2081F1
:1013400030E0092E02C0369527950A94E2F7217005
:101350003327042E01C0220F0A94EAF7822B4F5F35
:101360005F4F4530510531F70895BF92CF92DF921C
:10137000EF92FF920F931F93CF93DF938C01C09056
:10138000E101D090E201E090E301F090E40180916E
:10139000E5019091E601A091E701B091E801C82A2A
:1013A000D92AEA2AFB2ACFE1D0E0D701C6010C2EC8
:1013B00004C0B695A795979587950A94D2F780FDB6
:1013C00004C0219790F7B12C07C0BC2EB8018C2F18
:1013D0000E9402110197A9F38B2DDF91CF911F91EC
:1013E0000F91FF90EF90DF90CF90BF900895CF9333
:1013F000DF93EC010E94B509BE010E940211DF914A
:10140000CF9108951F93CF93DF93EB019091C70184
:10141000992321F0CB010E94F70913C0882349F0DA
:10142000CB010E94B509182F682FCE010E945E09DA
:1014300004C0CB010E948909182FBE01812F0E9490
:101440000211DF91CF911F9108951F93CF93DF93E6
:10145000C091E90116E08091EA01C81799F0D0E047
:101460001C9FF0011D9FF00D1124E551FE4F40819E
:10147000518162817381848195810E943E08219609
:10148000C770E9CFDF91CF911F91089540911B0262
:1014900050911C0260911D0270911E0280911F02EA
:1014A000909120020C943E08EF92FF920F931F93AD
:1014B000CF93DF938091200282958F7009F065C0F1
:1014C00080911D02882309F460C08091E901F090A9
:1014D000EA0110911B0200911C0260911E027091A2
:1014E0001F0291E01F3F09F090E0C0910001D091F0
:1014F0000101292F96E0E92E8F1509F446C06115E8
:10150000710521F00F3F21F030E003C031E001C050
:10151000322F90E030FD36C0E89EF001E99EF00DDC
:101520001124DF01A551BE4F11963C911197301344
:1015300029C03C91311326C012963C91129731116B
:1015400021C013964D915C911497461B570B4C1775
:101550005D07C0F4809120028F708061809320022B
:10156000E051FE4F80818F70806180838BE192E03B
:101570000E94BC07DF91CF911F910F91FF90EF90D8
:101580000C94250A01968770B7CFDF91CF911F91F8
:101590000F91FF90EF9008959F92AF92BF92CF92DC
:1015A000DF92EF92FF920F931F93CF93DF93CDB70C
:1015B000DEB761970FB6F894DEBF0FBECDBF8C01CA
:1015C00085E0F801DE011D9601900D928A95E1F704
:1015D000D8011296EC9090911B02E0911C02209190
:1015E0001E0230911F022115310531F0EF3F31F419
:1015F00081E09F3F19F403C081E001C080E0B82F73
:10160000B1709B2E80FD47C1D8014C9111965C9121
:1016100011971396AD90BC9014978BE1C82E82E081
:10162000D82EF0901D02B501621B730B20910001B2
:1016300030910101FF2009F4D9C080912002621786
:10164000730708F095C0282F207F09F052C05E1361
:1016500013C0491311C0FE2CE1100EC08F708061C1
:10166000809320020E94460AC6010E94BC07809116
:101670002002F80185834DC1AB2831F05F3F31F482
:1016800081E04F3F19F403C081E001C080E080FD9C
:1016900003C081E08E2502C080E090E0F82FF17059
:1016A000FF2E80FF1CC08091E9012091EA0136E005
:1016B000821709F40BC190E0389FF001399FF00DBB
:1016C0001124E551FE4F6181561306C06081461317
:1016D00003C06281E61203C001968770E9CFFE2C39
:1016E000EE2009F416C180912002816080932002CF
:1016F00054C05E1306C0491304C0E11002C0F801D3
:1017000099C0C8010E942708882361F1EE2051F199
:1017100020912002822F82958F7090E0029774F0C2
:1017200080911B0290911C0298878F831986BB863B
:10173000AA862C87CE0107960E94BC0786E0F80196
:10174000ABE1B2E001900D928A95E1F70E94540A54
:101750000E94460A0AC05E1711F1C8010E942708BC
:1017600081112CC0C8010E94BC07FF24F394D1C092
:10177000282F207F81F77A2DB98AA88A6E2D898932
:101780000E942F088BE192E00E94BC0786E0D60100
:101790001D928A95E9F70E94460AF12CBAC04913B6
:1017A000DCCFE110DACFF8018583C8010E94BC07C5
:1017B00086E0D6011D928A95E9F7ABC0EE2091F242
:1017C00020912002822F82958F7090E002970CF476
:1017D000B5CF80911B0290911C029A8389831B8252
:1017E000BD82AC822E83CE010196A6CF621773070D
:1017F00008F044C0FE2CEE2009F4B4CF5E1330C0D4
:1018000049132EC02091200220FD21C0822F8295F5
:101810008F70482F50E041155105C9F0F80125831C
:101820004F30510541F08F5F982F9295907F822F16
:101830008F70892B8583C8010E94BC0786E0F80160
:10184000ABE1B2E001900D928A95E1F73CC086E0F1
:10185000F801ABE1B2E001900D928A95E1F759C031
:10186000C8010E942708811169CF80912002816000
:1018700080932002C8010E94BC074BC07A2DB98A10
:10188000A88A6E2D89890E942F0886E0D6011D92B4
:101890008A95E9F718C0EE2009F464CFC8010E94C8
:1018A0002708F82E882309F45DCF86E0F801ABE124
:1018B000B2E001900D928A95E1F78BE192E00E94EF
:1018C0002D040E94540A0E94460A23C04D875E8759
:1018D0008D859E850E94F709292F22952F70223031
:1018E00028F49F7039F0811105C00BC0243028F412
:1018F0009F7049F4805E883020F0C8010E94BC07C8
:101900009F2CF92C06C0D80115969C91907F91F7D9
:10191000F8CF8F2D61960FB6F894DEBF0FBECDBF06
:10192000DF91CF911F910F91FF90EF90DF90CF90BB
:10193000BF90AF909F9008951F93CF93DF93CDB743
:10194000DEB72C970FB6F894DEBF0FBECDBF4F8326
:10195000588769877A878B879C87CE0107960E9474
:10196000CC0A8823D1F09F8188852A853B85232B4B
:1019700031F08F3F31F481E09F3F19F403C081E0E3
:1019800001C080E080FD47C04F81588569857A8518
:101990008B859C850E943E083EC086E0FE013796FE
:1019A000DE01119601900D928A95E1F7FF81E8859D
:1019B0006A857B856115710531F0EF3F31F481E077
:1019C000FF3F19F403C081E001C080E080FD23C027
:1019D0002091EA0130E0C901019687709927409172
:1019E000E90150E084179507F1F1F983EA837D83DB
:1019F0006C8396E0929FD001939FB00D1124A55166
:101A0000BE4FFE01319601900D929A95E1F78093B9
:101A1000EA010E94250A16E08091E9019091EA010D
:101A2000891771F1189FC001112485519E4F0E94A2
:101A3000CC0A882329F1E091E9011E9FF0011124CD
:101A4000E551FE4F4081518162817381848195818E
:101A50000E943E088091E90190E0019687709927E5
:101A60008093E901D9CF0E9408081092EA011092F0
:101A7000E901EBE1F2E086E0DF011D928A95E9F7EA
:101A80002C960FB6F894DEBF0FBECDBFDF91CF917D
:101A90001F910895809141028595859585950895BA
:101AA000809141028770089590914102977081E082
:101AB00009F480E008958091640208959091640291
:101AC000892B809364020895809590916402892304
:101AD00080936402089510926402089590916302C5
:101AE000892B8093630208958095909163028923E6
:101AF00080936302089510926302089580914202D8
:101B0000089508950C94810D0C94820D9091C20259
:101B100092FD08C090914202981721F080934202F2
:101B20000C94840D089580914202882329F010922C
:101B3000420280E00C94840D0895CF93DF93E091EE
:101B40000201F0910301809164028083E09102011F
:101B5000F0910301908180916302892B80838091B1
:101B60004202882381F0E0910201F091030190810B
:101B7000892B808380910201909103010E94E71FCD
:101B800081110E94930DC0910201D091030140E2A6
:101B900050E061E272E0CE010E942829892B69F0B1
:101BA00080E2FE01A1E2B2E001900D928A95E1F798
:101BB000CE01DF91CF910C94931FDF91CF910895C7
:101BC0000C94810D9091C20292FD10C098E0899F03
:101BD00090011124262B209341020E94C00880917D
:101BE00041028595859585950C94E00D0C94C0086F
:101BF0001092410280E00C94E00D2091410280950A
:101C0000822380934102982F977099F430E0482FF7
:101C1000082E000C550B2417350759F09091C2027D
:101C200092FD07C08595859585950E94E1080C94E5
:101C3000F80D08959091C20292FB222720F92817EF
:101C400069F080FB92F99093C2028091C102909159
:101C5000C2020E94680E82E00C94FD0D08958091EE
:101C6000C20282FB882780F991E089270C941A0E22
:101C700081E00C941A0E80E00C941A0E6FEF7FEF47
:101C800080E090E00C94672980E090E00E94432976
:101C900021E0893E9E4F09F020E0822F089582E0E6
:101CA00090E00C94352983E090E00C943529CF9393
:101CB00084E090E00E943529C82F82E290E00E94E3
:101CC00035292C2F30E0A901582BCA01CF91089556
:101CD000CF93C92F682F84E090E00E9449296C2F90
:101CE00082E290E0CF910C944929AB01BC018FE0D6
:101CF00090E00C945B29AB01BC0183E190E00C9473
:101D00005B2960E070E0CB010C947B0E60E070E03A
:101D1000CB010E94750E0C94810E69EE7EEF80E07F
:101D200090E00E94672960E082E090E00E944929EB
:101D300060E083E090E00E9449291092E501109252
:101D4000E6011092E7011092E80160E084E090E083
:101D50000E94492960E082E290E00E94492960E007
:101D600085E090E00E94492960E086E090E00E94D2
:101D700049296FEF87E090E00E94492940E050E058
:101D8000BA0188E090E00E945B2960E08DE090E07D
:101D90000E94492940E050E0BA0188E190E00E94A9
:101DA0005B2960E087E190E00E94492940E050E033
:101DB000BA018CE190E00E945B2960E070E080E273
:101DC00090E00E94672940E050E0BA0188E190E08D
:101DD0000E945B290C94860E0C948D0E682F8EE069
:101DE00090E00C9449290E944D2160936F027093FA
:101DF0007002809371029093720260936B027093F1
:101E00006C0280936D0290936E02089585B780688E
:101E100085BF85B7806885BF089581E008950C94DB
:101E20000D0F08950C94110F0C94110F0C94140FB6
:101E30000C94110F0C94180F0C94110F0E94060FA4
:101E40008EED91E10E947D1F0E941C0F0C941A0FD1
:101E50000E94120F0C94110F0E94F8110C94C503EC
:101E60000E9438210E94D6120E942C0F0E94641BEF
:101E70000C94160F5F926F927F928F929F92AF9207
:101E8000BF92CF92DF92EF92FF920F931F93CF9367
:101E9000DF93CDB7DEB72A970FB6F894DEBF0FBE3B
:101EA000CDBF0E94EB12C82E81110E94F30E35E6C1
:101EB000832E32E0932E00E010E0502E802F0E94FF
:101EC0001C125C01F401619071904F016826792623
:101ED00061147104B1F40F5F1F4F0330110569F7EE
:101EE0008FEF89838A831B820E9441218160782F32
:101EF0009D838C8349815A816B818D810E94E3038C
:101F00003AC08091730281FD0E942512D12CEE24EB
:101F1000E394F12CC3018E219F21892B29F10E948A
:101F20000F0F8823A9F0DE825F82AE20BF2081E000
:101F3000AB2809F480E088870E9441218160782FD6
:101F40009A8789874E815F8168858A850E94E3032D
:101F5000000F111FF801EB59FD4F80819181E82698
:101F6000F926F182E08207C0D394EE0CFF1CFDE05D
:101F7000DF12D0CFB0CF81E0C11001C080E02A963F
:101F80000FB6F894DEBF0FBECDBFDF91CF911F918A
:101F90000F91FF90EF90DF90CF90BF90AF909F9008
:101FA0008F907F906F905F9008950E943A0F0E94EB
:101FB000971B0E94F2140C94D803CF93DF930E94D6
:101FC0000711EC01811521E5920708F045C0811544
:101FD00030E5930708F094C0883E910528F5803ECF
:101FE000910508F0F8C0883A910570F4853A91059A
:101FF00008F07CC08130910509F475C008F4E8C090
:10200000049708F0E8C0E4C08F3B910508F0E0C0F9
:10201000C85AD0E0CC0FDD1FC35ADE4F0990D881DB
:10202000C02DCE019464D8C0811540E2940758F4C5
:10203000811551E0950708F0CEC08D3E910508F45A
:10204000C7C09065C9C0C11580E4D80708F4C0C0F6
:10205000DF70CE01906AC0C0811525E59207A8F413
:10206000811534E5930708F095C0811543E5940781
:1020700008F07BC0811552E5950708F061C0D82FA4
:10208000CC27CE01816F906AA7C0C11589E5D8071A
:10209000A0F4C11528E5D20708F082C0C11536E5C5
:1020A000D30708F095C08C2F0E949B118F7190E090
:1020B000D82FCC27CE0190628FC0C1154AE5D40736
:1020C00008F474C0CE0190568115904208F080C08B
:1020D0008D2F8F710E949B11DD27D0628F71AE0111
:1020E000582BCA0179C081E090E076C0C55AD0E093
:1020F000C557DE4F8881C82FD0E0CE0190646CC0F8
:1021000074E0969587957A95E1F7282F23703C2FF8
:10211000337081E090E002C0880F991F3A95E2F792
:102120009C68AC01522B9A019C2F9F7096959695B6
:1021300050E2959FE0011124C9018C2B9D2B4CC0CE
:102140008370992721E030E002C0220F331F8A9567
:10215000E2F79C2F9695969580E2989FE0011124D6
:10216000C22BD32BCE019C6837C08370992721E006
:1021700030E002C0220F331F8A95E2F79C2F96951C
:10218000969540E2949FE0011124C22BD32BCE01FF
:102190009A6822C0D82FCC27CE01846F906A1CC0C9
:1021A000DC2FCC27CE01806F906A16C08C2F8F70E9
:1021B0000E949B1194E0D695C7959A95E1F7CF7050
:1021C000D0E0DC2FCC27D0699E01282BC90104C0A8
:1021D00080E090E001C0CE01DF91CF91089527E229
:1021E000829FC0011124FC012DE0729FE00DF11DC2
:1021F0001124E60FF11DEE0FFF1FE852FF4F8591EE
:10220000949108950E94EF100E94DD0F0895823886
:10221000910569F1B0F48133910509F46DC048F47A
:102220008932910509F463C08A32910509F469C0C5
:1022300008958533910509F455C089339105B9F0A6
:102240000895833E910569F138F4803E9105B1F01F
:10225000823E910509F10895863E9105A9F1873ED8
:102260009105B9F1843E910509F064C023C0209125
:10227000C10220FD4FC021FD4DC008958091C102D3
:1022800080FD44C08091C20280FF44C08091C102A1
:1022900084FD42C083EE4DC08091C10282FF38C0F0
:1022A000F5CF8091C10282FD33C08091C20280FDD2
:1022B00031C0ECCF8091C20281FF32C08091C10257
:1022C00084FD2AC087EE35C08091C10283FF26C0FD
:1022D000F5CF8091C10283FD21C08091C20281FDB2
:1022E0001FC0ECCF8091C10285FD1CC01DC0809134
:1022F000C10285FD19C016C08091C10286FD16C0BD
:1023000017C08091C10286FD13C010C089E311C0BF
:1023100082EE0FC080EE0DC080E00BC086EE09C0DB
:1023200084EE07C089E205C085E303C08AE201C0EC
:1023300081E390E008959091C10292FF0DC0282F93
:102340002871283019F4877F846006C0282F2471F3
:10235000243011F48B7F886093FF0DC0282F2871E3
:10236000283119F4877E846106C0282F2471243116
:1023700011F48B7E88612091C20220FF0DC0382F9E
:102380003871383019F4877F816006C0382F317179
:10239000313011F48E7F886021FF0DC0282F287105
:1023A000283119F4877E816106C0282F21712131DF
:1023B00011F48E7E886194FD877E089580E00895F3
:1023C0000C943E0E0E94EB128FE39CE90197F1F70B
:1023D00000C000000E94EB1280E00E941C1280FFEF
:1023E00004C00E94E0110C948E2108950C94E21117
:1023F0000E94440E811102C00E94EC0E0E944F0EFA
:10240000809373020E94570E9093C2028093C10280
:102410000E94F6110E94530E682F70E080E090E059
:102420000E9460086091E1017091E2018091E301F6
:102430009091E4010C949808E82FF0E0EE0FFF1F54
:10244000E753FD4F808191810895089580EA8A9530
:10245000F1F7089500C008950C94261208950C9485
:102460002E120C942F120C942E120C943312F894FA
:10247000E82FE295EF70F0E031A1282F2F7081E076
:1024800090E001C0880F2A95EAF7982F9095932342
:1024900091A392A1892B82A378940895CF93DF937F
:1024A00084E90E94371284E30E94371285E30E9478
:1024B0003712CEE8D1E089918F3F11F00E94371298
:1024C00081E0CB39D807B9F7DF91CF910895BF925A
:1024D000CF92DF92EF92FF920F931F93CF93DF93F0
:1024E0008C01C62FD0E0CE0185569E4F6C01FC01B9
:1024F00090819F3F09F450C0B62EF894E92FE295E1
:10250000EF70F0E081A19F7021E030E001C0220F68
:102510009A95EAF7822B81A382A12095282322A3F2
:1025200078940E942A12EEE8F1E04BE951E021E0B4
:1025300030E0E12CF12C61916F3F89F0A62FA2953C
:10254000AF70B0E090968C9190E06F7002C095955E
:1025500087956A95E2F780FD02C0C90102C080E05C
:1025600090E0E82AF92A220F331F4E175F0719F768
:10257000F60180818F3F11F00E94371261E0E11473
:10258000F10409F460E08B2D0E942C12CC0FDD1FAA
:10259000C00FD11FF982E882DF91CF911F910F9177
:1025A000FF90EF90DF90CF90BF9008950E944E1261
:1025B00086E0E9ECF2E0DF01982F1D929A95E9F7A9
:1025C000E3ECF2E0DF011D928A95E9F783E00E94D7
:1025D00036130C943E03FF920F931F93CF93DF9318
:1025E00000D000D000D0CDB7DEB78E010F5F1F4FF7
:1025F00086E0F80111928A95E9F760E0C8010E942F
:10260000671261E0C8010E94671262E0C8010E947F
:10261000671246E050E0B80183EC92E00E9428295E
:10262000FF24F394009709F4F12C892B41F086E004
:10263000F801A3ECB2E001900D928A95E1F72F2DFD
:1026400043E069EC72E083EC92E00E9437130E9451
:1026500040038F2D26960FB6F894DEBF0FBECDBF78
:10266000DF91CF911F910F91FF9008950895FF92F0
:102670000F931F93CF93DF93F82E092F162FD72F89
:10268000C42F222349F081E0809376020E944121E9
:102690009093750280937402809176028823D9F01A
:1026A00080917402909175020E945921059798F0CB
:1026B000EF2DF02FA12FBD2F80E090E04C2F50E0A8
:1026C0008417950734F4219131912D933D93019610
:1026D000F7CF10927602DF91CF911F910F91FF906B
:1026E00008950E9446230E94300F0C9452230E94AA
:1026F00056230E94D50F0C9470230E94DF200E9465
:102700002D230E941E0F0E9471130E9477130E94B6
:10271000280FFBCF80917D0280FF06C060910901E8
:1027200070E0660F771F26C081FF04C06091090129
:1027300084E005C082FF07C06091090188E0689FBE
:10274000B001112417C090917C029923D1F06091BF
:102750000801961788F72091090188E0289F9001C9
:102760001124929FA001939F500D112470E0CA0183
:102770000E94A2286038710540F46115710519F4B2
:1027800006C068E070E0862F08958FE7089581E025
:10279000089580917D0280FF08C06091050170E07E
:1027A000759567957595679521C081FF06C0609105
:1027B000050170E07595679519C082FF04C06091AE
:1027C000050170E010C090917B02992399F060910F
:1027D00004019617A0F780910501899FC00111247B
:1027E00070E00E94A2286038710540F461157105FF
:1027F00019F406C061E070E0862F08958FE7089510
:1028000081E008958D3E21F40E948A13819504C0D1
:102810008E3E29F40E948A138093810208958F3E90
:1028200021F40E948A13819504C0803F29F40E94FC
:102830008A13809380020895893F19F40E94C91376
:1028400005C08A3F31F40E94C913819580938202AA
:1028500008958B3F21F40E94C913819504C08C3FD9
:1028600029F40E94C9138093830208959FE0980F72
:10287000983078F421E030E0A90102C0440F551FE0
:102880009A95E2F7CA0190917F02892B80937F028B
:1028900008958D3F21F480917D0281600BC08E3FB1
:1028A00021F480917D02826005C08F3F29F48091E0
:1028B0007D02846080937D0208958D3E39F490916D
:1028C000810297FF35C01092810259C08E3E29F4D3
:1028D000909181021916BCF32BC0909180028F3E1B
:1028E00029F497FF25C01092800249C0803F19F457
:1028F0001916CCF31DC090918202893F29F4191654
:10290000BCF4109282023BC08A3F19F497FF10C0BA
:10291000F8CF8B3F39F49091830297FF09C0109252
:1029200083022DC08C3F21F4909183021916BCF3D1
:102930009FE0980F983080F421E030E0A90102C0B8
:10294000440F551F9A95E2F7CA01809590917F0236
:10295000892380937F0213C08D3F21F480917D02F3
:102960008E7F0BC08E3F21F480917D028D7F05C04C
:102970008F3F29F480917D028B7F80937D0280912F
:102980008002811106C080918102811102C01092E3
:102990007C0280918202811106C0809183028111A4
:1029A00002C010927B0208950E9441212091800272
:1029B000211104C020918102222321F090937A02F8
:1029C0008093790220918202211104C02091830218
:1029D000222321F090937802809377028EE792E091
:1029E0000C94AD1FEF92FF920F931F93CF93DF9341
:1029F00000D000D000D0CDB7DEB786E0EEE7F2E041
:102A0000DE01119601900D928A95E1F7E090800227
:102A1000F090810200918202109183021092800254
:102A2000109281021092820210928302E11003C080
:102A3000FF2009F45DC08091790290917A020E9492
:102A40005921AC0190917C02992339F020910A011F
:102A500030E02417350758F04BC020910B018AE075
:102A6000289F900111242417350718F041C09F3F7B
:102A700019F09F5F90937C02EE2061F00E948A1310
:102A80001E1414F09FEF01C091E0989F902D112427
:102A900090938002FF2061F00E948A131F1414F0AB
:102AA0009FEF01C091E0989F902D11249093810297
:102AB000309180023323E1F0209181022223C1F082
:102AC00045EB3403C0011124992319F0909380023F
:102AD00003C081E08093800235EB2303C001112401
:102AE000992319F09093810203C081E080938102C1
:102AF000011103C0112309F45DC080917702909108
:102B000078020E945921AC0190917B02992339F0FF
:102B10002091060130E02417350758F04BC0209172
:102B200007018AE0289F900111242417350718F027
:102B300041C09F3F19F09F5F90937B02002361F09B
:102B40000E94C913101614F09FEF01C091E0989FE6
:102B5000902D112490938202112361F00E94C913D9
:102B6000111614F09FEF01C091E0989F902D112451
:102B700090938302309182023323E1F0209183020B
:102B80002223C1F045EB3403C0011124992319F02D
:102B90009093820203C081E08093820235EB23038D
:102BA000C0011124992319F09093830203C081E09E
:102BB000809383028091800281110BC080918102F9
:102BC000811107C080918202811103C0809183022C
:102BD00081110E94D414EB82FC820D831E8386E057
:102BE000FE013196AEE7B2E001900D928A95E1F7D1
:102BF00026960FB6F894DEBF0FBECDBFDF91CF9102
:102C00001F910F91FF90EF900895EEE7F2E086E0BC
:102C1000DF011D928A95E9F710927C0210927B02E7
:102C200010927D020895EF92FF920F931F93CF931E
:102C3000DF938B01682F11110AC0442329F0E82F7C
:102C4000F0E0E95DFC4F6491762F862F75C0212F4F
:102C500030E0E82FF0E0442321F0E95DFC4FE491FF
:102C6000F0E046E0049FC0011124CFEFD0E0BE01A8
:102C70000E948E284BEA4603C001479F900D112405
:102C8000800F911D800F911D982F990F890FAE0114
:102C9000421B530B4E9FD0014F9FB00D5E9FB00D56
:102CA00011249B2F189FA0011124452F55278E0119
:102CB000041B150B0E9FA0010F9F500D1E9F500D62
:102CC00011247E01E81AF108E29E8001E39E100DB6
:102CD000F29E100D1124212F3327C21BD30BCE9F40
:102CE0009001CF9F300DDE9F300D112462307105B1
:102CF000A9F048F46115710569F061307105C9F4F6
:102D00008B2F752F0DC06430710581F058F066303F
:102D1000710579F47E2F8B2F932F0DC0832F7B2F7E
:102D20009E2F09C08E2F7B2F952F05C08E2F732FBE
:102D300002C07E2F852F692FDF91CF911F910F91B8
:102D4000FF90EF90089541E00E94131608950895B2
:102D50000E94A3160895CF93DF93762FE901682F81
:102D6000842F0E94A816798368838A83DF91CF918C
:102D700008958091CF02282F269530E02115310546
:102D800019F48170826005C02532310524F081700C
:102D900088648093CF02089588E090E00C943D29E8
:102DA000CF92DF92EF92FF926B017C010E94B916E5
:102DB000B701A60188E090E0FF90EF90DF90CF9000
:102DC0000C945B29EFECF2E083E0808311828FEFBB
:102DD00082838383148260817181828193810C94C8
:102DE000D0168091CF0280FF02C08695089580E0C2
:102DF00008959091D302933018F49F5F9093D3027B
:102E0000882351F06091CF027091D0028091D1025D
:102E10009091D2020C94D016089581E00C94F9168A
:102E20009091D302992319F091509093D302882363
:102E300051F06091CF027091D0028091D1029091B7
:102E4000D2020C94D016089581E00C94101770E013
:102E50000C94141D609110018091CF0280FF0AC074
:102E600080910F0123E0829FC00111248C529D4F5D
:102E70000C9427178091110190911201891780F706
:102E8000E82FF0E09F01220F331FE20FF31FEC52F7
:102E9000FD4F1182108212828F5FF0CF9091CF028E
:102EA00090FF16C09091110120911201921770F4B9
:102EB000E92FF0E0DF01AA0FBB1FEA0FFB1FEC5266
:102EC000FD4F8183608342839F5FF0CF0C942A176C
:102ED0000895CF93DF9300D01F92CDB7DEB79091C6
:102EE000CF0290FF0AC09E012F5F3F4F0E94AB169A
:102EF0004B8169818A810E944E170F900F900F902D
:102F0000DF91CF910895CF93DF93EC01EC81F0E056
:102F1000EE5DFD4F4491EFECF2E0628181810E9411
:102F200069178C818F5F8C83DF91CF910895CF9348
:102F3000DF93EC01EFECF2E0438162818C810E942F
:102F400069178C818F5F8C83DF91CF9108950F93E8
:102F50001F93CF93DF9300D01F92CDB7DEB78C01C4
:102F60008091840281110AC09E012F5F3F4F4FEF75
:102F70006FEF0E94AB168A8180938402F8018481EE
:102F8000813051F028F0823061F4409184020AC00F
:102F90008091840240E007C06091840240E080E0BC
:102FA00003C040E080E060E00E944E17F801848199
:102FB00090E0019663E070E00E94A22884830F9065
:102FC0000F900F90DF91CF911F910F910895AF92C5
:102FD000BF92CF92DF92EF92FF920F931F93CF9306
:102FE000DF9300D01F92CDB7DEB7182FF62E042F37
:102FF000E22E9091CF0290FF6DC0E92FE695AE2FA3
:10300000B0E0A256BE4F8C9180938E029E7F92308C
:1030100061F49E012F5F3F4F812F0E94AB164B81C1
:1030200069818A810E944E1743C0823019F4009151
:10303000D2023EC0863019F41091D00239C08930D6
:10304000D9F38931A9F5E9518E2F8170D82EE695F3
:10305000F0E0EE5DFC4FA590B490C12CBB246091D4
:103060001301C61618F52C2D30E0A29EC001A39EB8
:10307000900DB29E900D112470E00E948E28812F39
:10308000D11002C0860F01C0861B90911101290F3B
:10309000311DA901440F551F240F351F2C523D4FE0
:1030A000402F6F2D0E94AB16C394D9CF0E942A17D0
:1030B0001093D002F092D1020093D202EE2051F090
:1030C0006091CF027091D0028091D1029091D20292
:1030D0000E94D0160F900F900F90DF91CF911F910B
:1030E0000F91FF90EF90DF90CF90BF90AF90089539
:1030F000EFECF2E09181282F4381628188E0890F13
:103100000C94E71781E00C947818EFECF2E09181D1
:10311000282F4381628188EF890F0C94E71781E0A3
:103120000C948518EFECF2E0628128E0620F08F45D
:103130006FEF282F438181810C94E71781E00C9475
:103140009218EFECF2E0628128E0621B08F460E084
:10315000282F438181810C94E71781E00C94A118FA
:10316000EFECF2E0438128E0420F08F44FEF282F04
:10317000628181810C94E71781E00C94B018EFEC28
:10318000F2E0438128E0421B08F440E0282F6281EE
:1031900081810C94E71781E00C94BF1820E00C9417
:1031A000E717FF920F931F93CF93DF93EC01F12C5E
:1031B0000FEF10E060911301F616F0F48091110109
:1031C0002F2D30E0280F311DC901880F991F280FBE
:1031D000391F2C523D4F70E0C8010E94A228962F43
:1031E0008C814091D2026091D102F99E800D112410
:1031F0000E94AB16F394DECF0E942A179A818C812D
:1032000090FF02C08F5F01C081508C83DF91CF910E
:103210001F910F91FF900895AF92BF92CF92DF92CE
:10322000EF92FF920F931F93CF93DF93FC01828164
:1032300080FF02C00FEF01C001E010E045E0A42EC6
:1032400080911301181708F043C080911101C12E1D
:10325000D12CE601C80FD11DCE01880F991FC80FD0
:10326000D91FCC52DD4F198218821A8234E0E32E26
:10327000F12CB12C809186028B0D86302CF06A2DBA
:103280000E948028892F05C087FF03C090911301F9
:10329000890F082E000C990BC816D90691F480915D
:1032A000D2028E9DA0018F9D500D112455954795FA
:1032B000559547959E016091D1028091D0020E9460
:1032C000AB16B00EF1E0EF1AF108A1F61F5FB8CF10
:1032D0000E942A1780918602013031F4811102C0C8
:1032E00080911301815007C090E001966091130115
:1032F00070E00E94A22880938602DF91CF911F91F7
:103300000F91FF90EF90DF90CF90BF90AF90089516
:10331000CF938091110190911201891770F4E82FD9
:10332000F0E09F01220F331FE20FF31FEC52FD4F1D
:103330001182108212828F5FF0CFC0E06091130182
:10334000C617C0F5EC2FF0E070E0CF010E94A22874
:1033500020911101820F20918502022E000C330B67
:1033600090E0E217F307CCF020910E01022E000C42
:10337000330B2E173F078CF09C01220F331F820F57
:10338000931F9C012C523D4F4091D2026091D1027B
:103390008091D0020E94AB160BC0FC01EE0FFF1F04
:1033A0008E0F9F1FFC01EC52FD4F11821082128282
:1033B000CF5FC4CF0E942A1720910D018091850212
:1033C000820F8093850290910E01920F90930E01CF
:1033D00019165CF4082E000C990B4091130150E073
:1033E00041505109841795071CF0219520930D0138
:1033F000CF9108958F929F92AF92BF92CF92DF921A
:10340000EF92FF920F931F93CF93DF938C01FC01F8
:103410004481C42FD0E09E01DE010E94E6289B017A
:10342000AC010E94FC286B017C01E0E2F0E0EC1BA7
:10343000FD0BA5E5B0E09B01AC010E94FC284B010F
:103440005C019F01DF010E94DE289B01AC010E940C
:1034500007299B01AC012C0D3D1D4E1D5F1DC501B3
:10346000B4010E94B628C22FD22F2A3228F4F3E0EA
:103470002F9F900111240DC025E530E02C1B310950
:10348000C901880F991F280F391F37FF02C02F5F0E
:103490003F4F35952795C22FC095F12C85E5E82E35
:1034A000ED1A80911301F816C8F4F1FC02C08E2DBC
:1034B00001C08D2F909111012F2D30E0290F311D6A
:1034C000A901440F551F240F351F2C523D4F4C2F7F
:1034D0006091D1020E94AB16F394E3CF0E942A17A9
:1034E000F8018481811102C091E003C0803219F497
:1034F0009FEF90930C0190910C01890FF801848348
:10350000DF91CF911F910F91FF90EF90DF90CF90BF
:10351000BF90AF909F908F9008950F931F93CF937C
:10352000DF93EC0100E010E080911301282F30E0E0
:103530000217130724F5909111019801290F311DED
:10354000A901440F551F240F351F2C523D4F86955E
:1035500090E04C81081719071CF4442331F002C095
:10356000411103C04091D20201C040E06091D102FC
:103570008091D0020E94AB160F5F1F4FD5CF0E94E3
:103580002A178C8190E00196817099278C83DF91B6
:10359000CF911F910F910895EFECF2E080818E7F23
:1035A000808360817181828193810E94D016109204
:1035B0008F022FEF80E792E0215080409040E1F7AA
:1035C00000C000000C942A176091CF02669570E04D
:1035D0004BE050E084E191E00E941B29892B19F413
:1035E00081E080938F020E94412190938802809312
:1035F000870208959091CF0290FF35C0917081119C
:1036000002C0926006C0853210F0986402C0880F34
:10361000982B9093CF02662351F06091CF02709166
:10362000D0028091D1029091D2020E94D016609176
:10363000CF02669570E04BE050E084E191E00E949B
:103640001B29892B19F010928F0202C00E94E41AE4
:1036500081E080938A024091D2026091D1028091F0
:10366000D0020C94CE180895682F9091CF029695B1
:1036700081E0890F853208F081E00C94FA1A81E02C
:103680000C94341B682F9091CF0296958FEF890F81
:1036900009F484E20C94FA1A81E00C94421B61E074
:1036A0000C94FA1AEFECF2E08081816080838695B9
:1036B0000C944F1B8091CF0280FD0C94CC1A0C947B
:1036C000521B60E00C94FA1A80918D0281112EC079
:1036D0000E94440E811104C00E94EC0E0E94E2166A
:1036E0000E94CC166093CF027093D0028093D102D7
:1036F0009093D2026E7F61F40E94E2160E94CC1673
:103700006093CF027093D0028093D1029093D20243
:103710000E94B91610928F028091CF0280FF03C0E1
:1037200086950E94611B81E080938D0208950F931E
:103730001F93CF93DF9380918F02882309F485C074
:1037400080918E02E091CF02E695E81BE09389021A
:10375000823049F4F0E0E25EFD4FE491CE2FD0E0FC
:1037600003E817E149C0863049F4F0E0E55EFD4F1B
:10377000E491CE2FD0E007E917E13EC0893051F443
:10378000E695F0E0E85EFD4FE491CE2FD0E001ED4C
:1037900018E132C08F3051F4E695F0E0EB5EFD4F5A
:1037A000E491CE2FD0E00CE019E126C0853149F438
:1037B000F0E0EE5EFD4FE491CE2FD0E008E819E195
:1037C0001BC0883181F0833239F4E0E1F2E0C59129
:1037D000D49107EA17E110C0843251F4C4EFD1E06C
:1037E0000DE81AE109C0C8E2D0E00AEF19E104C00F
:1037F000C0EDD7E007EA16E180918A02882361F0E4
:1038000010928A020E94412190938802809387023D
:1038100010928C0210928B020E944121E09187024B
:10382000F09188028E1B9F0B8F3F9F4770F4EC0F27
:10383000FD1FF0938802E093870287E892E0F80189
:10384000DF91CF911F910F910994DF91CF911F913B
:103850000F910895882311F0FA0101C0FB0109942A
:10386000CF93DF93C82FD62F0E94F1168C1740F00C
:103870000E94F1168D1720F4DF91CF910C943F1B1D
:103880008C2FDF91CF910C944F1B1F93CF93DF931D
:10389000FB0112811111C3C0EC010E945B0D827209
:1038A000CD3CFCE5DF0709F49AC0A8F5C73CECE580
:1038B000DE0709F476C0A8F4C43C9CE5D90709F4F6
:1038C0005FC028F4C33CDC4509F457C054C0C53C74
:1038D0009CE5D90709F459C0C63CDC4509F45CC035
:1038E0004AC0CA3CFCE5DF0709F46AC050F4C83C92
:1038F000ECE5DE0709F45AC0C93CDC4509F45BC0BD
:103900003AC0CB3C9CE5D90709F45FC0CC3CDC4510
:1039100009F460C030C0C23DFCE5DF0709F46FC0A8
:1039200088F4CF3C9CE5D90709F460C008F45CC07A
:10393000C03DFCE5DF0709F45CC0C13DDC4509F48E
:103940005BC019C0C53D9CE5D90709F460C050F4BF
:10395000C33DFCE5DF0709F455C0C43DDC4509F46F
:1039600054C009C0C63D9CE5D90709F455C0CE3501
:10397000DD4509F454C011E052C00E945A1B4FC0EB
:103980004CE45BE16FE37BE104C04FE35BE16CE49B
:103990007BE10E942A1C43C04FE858E162E878E1CD
:1039A000F8CF42E858E16FE878E1F3CF4DEA58E10B
:1039B0006EE978E1EECF4EE958E16DEA78E1E9CFC2
:1039C0004BEC58E16CEB78E1E4CF4CEB58E16BEC5D
:1039D00078E1DFCF44E257E16DE077E1DACF4DE007
:1039E00057E164E277E1D5CF81E017C065E082E07E
:1039F00010C068E086E00DC06EE089E00AC064E1B6
:103A00008FE007C067E185E104C088E106C062E29B
:103A100089E10E94301C03C083E20E944F1B812F6A
:103A2000DF91CF911F910895849A21B32F7E31B3F6
:103A300030614FB7F894FC01CB01880F991F680FD4
:103A4000791F6E0F7F1FE617F70789F0819198E0C5
:103A500031BB000000C087FF21BB880F000000C001
:103A600000C000C021BB00C09A9591F7ECCF4FBFBA
:103A70008FE594E00197F1F700C000000895CF931F
:103A8000DF93EC01FB018281882309F43CC1C4303F
:103A9000FDE5DF0760F4CB3F9CE5D90788F49E0184
:103AA00022503C452431310508F02EC109C0C236F0
:103AB000EDE5DE0729F0C63AFDE5DF0709F024C190
:103AC0000E94570E9093C2028093C102C1318CE5CF
:103AD000D80709F4C6C008F042C0C930ECE5DE07DB
:103AE00009F49BC000F5C5308CE5D80709F485C002
:103AF00078F4C330ECE5DE0709F478C008F07AC04A
:103B0000C230DC4509F0F5C08091C1028160EFC090
:103B1000C7309CE5D90709F478C008F07AC08091D5
:103B2000C1028061E4C0CD30FCE5DF0709F487C045
:103B300058F4CB309CE5D90709F479C008F07BC074
:103B40008091C10288606FC0CF30FCE5DF0709F4C7
:103B500080C008F082C08091C102877FC8C0CE3F7C
:103B60009CE5D90709F471C000F5C531FCE5DF0714
:103B700009F485C068F4C3319CE5D90709F475C020
:103B800008F095C00E9408088091C1028F77AFC0ED
:103B9000CC3FFCE5DF07A9F108F054C0CB3FDC4582
:103BA00009F0A7C08091C20240C0C230EDE5DE0737
:103BB00009F489C058F4C1158DE5D80709F45AC035
:103BC00008F069C08091C20282602FC0C236EDE564
:103BD000DE0709F47CC0C63AFDE5DF0709F481C0C1
:103BE000C330DD4509F085C080E06EC08091C10220
:103BF00082607DC08091C10216C08091C102886040
:103C000076C08091C20282604FC08091C102806202
:103C10006EC08091C10280646AC00E9408088091D1
:103C2000C102806864C0846062C081603DC08091D0
:103C3000C1028E7F5CC08091C1028D7F58C080918F
:103C4000C10216C08091C20218C08091C2028D7F4D
:103C50002BC08091C1028F7E4AC08091C1028F7DAE
:103C600046C08091C1028F7B42C08091C102877F94
:103C70008B7F3DC08091C2028D7F8E7F15C0809169
:103C8000C10282FB222720F991E0922790FB82F962
:103C900090FB83F92CC08091C202982F909591706F
:103CA0008E7F892B90FB81F98093C20222C00E94F3
:103CB00008088091C10287FB222720F991E0922712
:103CC00090FB87F914C081E00E94EE0E12C0809133
:103CD000C10284FB222720F991E0922790FB84F90E
:103CE00006C08091C102982F909590FB80F9809337
:103CF000C1028091C1029091C2020E94680E0E948E
:103D0000080880E001C081E0DF91CF910895CF9352
:103D1000DF9386319C4541F5EB010E945B0D982FA6
:103D20008A812091020130910301882379F09A7AE7
:103D300081E009F480E080939002911102C069E271
:103D400001C065E3C9010E947D200AC080919002F4
:103D5000811102C069E201C065E3C9010E948820A7
:103D60000E949D0D80E001C081E0DF91CF91089518
:103D70000F931F93CF93DF93C42FD22FFC01828127
:103D80008823C9F0409393020E94412190939202AC
:103D90008093910280E28C0F883008F057C0C77082
:103DA00081E001C0880FCA95EAF7DF91CF911F919A
:103DB0000F910C94650580919302481330C0809157
:103DC0009102909192020E945921883C910538F508
:103DD00010E21D0FCD17B9F080E28C0F883040F44F
:103DE000C77081E001C0880FCA95EAF70E946C0590
:103DF000183028F581E09D2F977001C0880F9A95A3
:103E0000EAF70E946505802F0E945C051830F0F4E7
:103E1000D77081E001C0880FDA95EAF70AC080E226
:103E20008C0F883098F4C77081E001C0880FCA9564
:103E3000EAF7DF91CF911F910F910C946C05802FC1
:103E4000DF91CF911F910F910C945C05DF91CF9181
:103E50001F910F9108950F939C01CB01243F4CE5D6
:103E6000340731F188F4293DFCE53F07D9F02A3DBC
:103E70004CE5340779F1283D3C45A9F506E221EEF1
:103E800041EE68ED7CE52BC0263FFCE53F07E1F005
:103E9000A8F0273F3C4539F507E225EE46EE67EFEF
:103EA0007CE51DC007E225EE45EE69ED7CE517C017
:103EB00006E221EE40EE64EF7CE511C007E225EE5C
:103EC00044EE65EF7CE50BC006E221EE42EE66EFC4
:103ED0007CE505C008E221E045EE6AED7CE50E9444
:103EE000B81E80E008C0FC018281882319F010927E
:103EF000930201C081E00F9108959093C5018093D2
:103F0000C401089590939902809398020895E091D6
:103F10009802F0919902309721F00190F081E02D04
:103F2000099480E00895E0919802F0919902309709
:103F300099F020912B01222359F02091C10227FFF3
:103F400007C0DC012C9111962C93119726E02C933D
:103F50000280F381E02D09940895E0919802F09198
:103F60009902309739F022E0DC012C930480F5812E
:103F7000E02D099408952091960230919702281718
:103F8000390771F09093970280939602E09198021E
:103F9000F0919902309721F00680F781E02D099485
:103FA000089520919402309195022817390771F0F5
:103FB0009093950280939402E0919802F091990277
:103FC000309721F00084F185E02D09940895FC01DB
:103FD000329680912B01882331F08091C10287FFB6
:103FE00002C09EE101C096E080E0915028F021914E
:103FF0002223D9F38F5FF9CF0895662351F12091E1
:104000002B012223E9F02091C10227FF19C0462F7E
:104010004695469546954E31E0F4677021E030E0D4
:1040200002C0220F331F6A95E2F7FC01E40FF11D75
:10403000828190E02823392381E0232B69F409C091
:10404000FC01329608962191621729F0E817F907CA
:10405000D1F780E0089581E008959C01FC0132963B
:104060009FEF80E04191461789F09F3F19F441117D
:1040700001C0982F8F5F8630A9F79F3F39F0F90173
:10408000E90FF11D97FDFA956283089508959C014B
:104090002A5F3F4FFC014281461301C01282019604
:1040A00082179307B9F70895262F2695269526950A
:1040B0002E3168F4FC01E20FF11D677021E030E061
:1040C00001C0220F6A95EAF78281282B2283089586
:1040D000262F2695269526952E3170F4FC01E20FA9
:1040E000F11D677021E030E001C0220F6A95EAF708
:1040F0002095828128232283089520912B01222359
:1041000029F02091C10227FD0C9454200C942D20FD
:1041100020912B01222329F02091C10227FD0C942C
:1041200068200C94472020912B01FC013296222319
:1041300031F08091C10287FF02C08EE101C086E0AC
:10414000DF011D928A95E9F7089508950C94A52042
:1041500083E080939A020C94A620811102C081E032
:1041600001C082E080939A020C94A6200C94AD20AA
:1041700081E080939A020C94A6200C94B8200895B4
:104180000C94BF200C94C0200C94BF200C94BF2032
:104190000C94BF20CF930E94C6200E94EB120E9475
:1041A000C420C0E08C2F0E941C12892B29F4CF5F01
:1041B000C330C1F780E001C081E0CF910895089538
:1041C0001F920F920FB60F9211248F939F93AF936C
:1041D000BF9380919B02811113C08091E302909163
:1041E000E402A091E502B091E6024196A11DB11D45
:1041F0008093E3029093E402A093E502B093E60279
:10420000BF91AF919F918F910F900FBE0F901F9014
:1042100018958091EB02843031F10E94AB0310922B
:104220009B0220E488E190E00FB6F894A895809373
:1042300060000FBE2093600083B7817F846083BFDE
:1042400083B7816083BF7894889583B78E7F83BF5F
:104250000FB6F894A8958091600088618093600003
:10426000109260000FBE08950E9408080C94AF03DE
:1042700082E084BD93E095BD9AEF97BD80936E0078
:1042800008952FB7F8948091E3029091E402A091F1
:10429000E502B091E6022FBF08952FB7F894609120
:1042A000E3027091E4028091E5029091E6022FBF53
:1042B00008959C014FB7F8948091E3029091E40235
:1042C000A091E502B091E6024FBF821B930B0895C7
:1042D00078941F920F920FB60F9211248F939F9391
:1042E000AF93BF938091E3029091E402A091E50225
:1042F000B091E6020196A11DB11D8093E302909357
:10430000E402A093E502B093E602BF91AF919F91C2
:104310008F910F900FBE0F901F90189587E797E72A
:1043200090930108809300089AE088E10FB6F89412
:10433000A895809360000FBE90936000FFCF80919E
:10434000BF020895089522E02093E9002FEF3091F5
:10435000E800215035FD06C035ED3A95F1F7000033
:104360002111F5CF2091E80025FF0BC040E050E07F
:1043700066E070E00E94E2238091E8008E778093EF
:10438000E8000895CF93DF9320912B01222339F089
:104390002091C10227FF03C060E222E002C068E072
:1043A00021E02093E9002FEF3091E800215035FD06
:1043B00006C035ED3A95F1F700002111F5CF2091B7
:1043C000E80025FF1DC0EC0180912B01811105C083
:1043D00040E050E068E070E003C070E040E050E092
:1043E000CE010E94E2238091E8008E778093E8005E
:1043F00080E2FE01AFE9B2E001900D928A95E1F70B
:10440000DF91CF91089580939C0270939E026093F8
:104410009D028091EB02843001F582E08093E900F7
:104420008FEF9091E800815095FD06C095ED9A952B
:10443000F1F700008111F5CF8091E80085FF0DC0F4
:1044400040E050E063E070E08CE992E00E94E223FB
:104450008091E8008E778093E8000895BC0184E0A5
:104460000C940322BC0183E00C9403228091EA02A5
:10447000811109C00E9473250E94D0258091E2001D
:1044800084608093E20008951092EA0208950C94EB
:10449000BD206091E70281E0611101C080E00C94D1
:1044A000A8209091EB0281E0943009F080E06091C7
:1044B000E7020C94AD2042E061EC81E00E94EC2424
:1044C00042E261EC82E00E94EC249091EB0281E0F8
:1044D000943009F080E06091E7020C94B62080915E
:1044E000ED02833009F461C030F4813071F0823024
:1044F00009F49AC008958A3009F486C08B3009F413
:104500006CC0893009F0A8C020C08091EC02813ACB
:1045100009F0A2C08091E800877F8093E800809135
:10452000F0029091F102892B21F460E28FE992E090
:1045300003C060E080E090E070E00E942D24809154
:10454000E8008B778093E80008958091EC02813237
:1045500009F082C08091F0029091F102029708F078
:104560007BC08091E800877F8093E8008091E8001D
:1045700082FD05C08091EB028111F8CF6DC02091C2
:10458000F3008091F20090E0922B029731F4809139
:10459000F100813011F0863021F48091F100809398
:1045A000BF028091E8008B7753C08091EC02813A82
:1045B00009F052C08091F0029091F102892B09F02C
:1045C0004BC08091E800877F8093E8008091E800ED
:1045D00080FFFCCF80912B0136C08091EC028132AC
:1045E000D9F58091F0029091F102892BA9F5809183
:1045F000E800877F8093E8000E9421258091EE02E9
:1046000080932B010C9408088091EC02813221F5F3
:104610008091E800877F8093E8000E9421258091A7
:10462000EF028093C00208958091EC02813AA1F4D8
:104630008091E800877F8093E8008091E80080FF08
:10464000FCCF8091C0028093F1008091E8008E77CA
:104650008093E8000C942125089584B7877F84BF58
:104660000FB6F894A89580916000886180936000EF
:10467000109260000FBE90E080E80FB6F89480932F
:104680006100909361000FBE0C94B8200E947325C6
:104690000E94D025E2EEF0E08081846080837894EF
:1046A0000C9465288FE191E00C94821F8091EB02BD
:1046B0008530A9F48091EB02853079F40E940921BC
:1046C0008091E9028823B1F30E94CA20882391F3E4
:1046D0000E94CC230E940808EDCF0C943421089549
:1046E00008950C947323292F332723303105C9F003
:1046F00060F42130310581F02230310509F044C0E9
:104700008BE390E027E534E043C021323105E1F04E
:104710002232310549F138C082E190E022E934E0EB
:1047200037C099278130910549F028F0029761F54B
:10473000E7E2F4E005C0E3E5F4E002C0E7E3F4E01B
:10474000849190E09F0124C06115710541F06130B2
:104750007105D1F489E090E022E834E019C089E0E5
:1047600090E029E634E014C06115710541F0613034
:10477000710551F486EB90E024EA34E009C080E44E
:1047800090E02AE535E004C080E090E020E030E0F1
:10479000FA0131832083089580E189BD82E189BDDA
:1047A00009B400FEFDCF8091D8008F7D8093D800A2
:1047B0008091E00082608093E0008091E00081FDC4
:1047C000FCCF0895CF92DF92EF92FF920F931F9349
:1047D000CF93DF93EC018B017A010E944025811178
:1047E00033C0E114F10439F0F70180819181081B95
:1047F000190BC80FD91FC12CD12C0115110519F1A6
:104800008091E80085FD16C08091E8008E77809346
:10481000E800E114F10449F0F70180819181C80EAC
:10482000D91ED182C08285E00FC00E944025882316
:1048300021F30AC089918093F10001501109FFEF23
:10484000CF1ADF0ADACF80E0DF91CF911F910F916D
:10485000FF90EF90DF90CF9008952091F202309179
:10486000F3022617370748F06115710539F42091D6
:10487000E8002E772093E80001C0B901FC0120E098
:104880006115710579F18091EB028823F1F1853092
:10489000F1F18091E80083FD3CC08091E80082FD49
:1048A0002EC08091E80080FFEBCF2091F300809133
:1048B000F20090E0922B6115710551F0883091055E
:1048C00038F421912093F100615071090196F3CFE2
:1048D00021E0089709F020E08091E8008E7780932E
:1048E000E800CECF2111CFCF0AC08091EB02882300
:1048F00061F0853061F08091E80083FD0AC080910D
:10490000E80082FFF2CF80E0089582E0089583E01E
:10491000089581E008952091F2023091F302261764
:10492000370748F06115710539F42091E8002E77BA
:104930002093E80001C0B901FC0120E06115710578
:1049400091F18091EB02882309F440C0853009F48D
:104950003FC08091E80083FD3DC08091E80082FD6A
:104960002FC08091E80080FFE9CF2091F300809173
:10497000F20090E0922B6115710559F08830910595
:1049800040F424912093F100319661507109019611
:10499000F2CF21E0089709F020E08091E8008E77BF
:1049A0008093E800CBCF2111CCCF0AC08091EB02DD
:1049B000882361F0853061F08091E80083FD0AC0B2
:1049C0008091E80082FFF2CF80E0089582E00895B0
:1049D00083E0089581E00895982F973068F59093CB
:1049E000E900981739F07091EC002091ED0050919A
:1049F000F00003C0242F762F50E021FD02C09F5FFE
:104A0000ECCF3091EB003E7F3093EB003091ED0026
:104A10003D7F3093ED003091EB0031603093EB003F
:104A20007093EC002093ED005093F0002091EE0085
:104A300027FDE5CF80E008958F708093E90081E045
:104A400008958091EC0287FF11C08091E80082FDFB
:104A500005C08091EB028111F8CF11C08091E80070
:104A60008B770BC08091EB02882349F08091E8009E
:104A700080FFF8CF8091E8008E778093E80008955A
:104A80002091E4003091E50095E64091EC00842F00
:104A9000817040FF23C08091E80080FD1DC080919F
:104AA000EB02882399F0853099F08091EB0085FD29
:104AB00011C04091E4005091E5002417350729F317
:104AC000915011F09A01E1CF84E0089582E00895B9
:104AD00083E0089581E0089580E008954091E80022
:104AE00042FFDDCF08950E94E1250E94E925E0EE16
:104AF000F0E0808181608083E8EDF0E080818F7755
:104B0000808319BCA7EDB0E08C918E7F8C9380815F
:104B10008F7E80831092EA0208950F931F93CF93A4
:104B2000DF930E94E1250E94E925C8EDD0E088814D
:104B30008F77888388818068888388818F7D888348
:104B400019BC1092EB021092E7021092E902109247
:104B5000E80200EE10E0F80180818B7F808388817D
:104B60008160888342E060E080E00E94EC24E1EE16
:104B7000F0E080818E7F8083E2EEF0E080818160D2
:104B80008083808188608083F80180818E7F80832C
:104B9000888180618883DF91CF911F910F91089563
:104BA000E8EDF0E080818F7E8083E7EDF0E08081AA
:104BB0008160808384E082BF81E08093EA020C946C
:104BC0008D25E8EDF0E080818E7F80831092E200F9
:104BD00008951092DA001092E10008951F920F924A
:104BE0000FB60F9211242F933F934F935F936F93C0
:104BF0007F938F939F93AF93BF93EF93FF93809196
:104C0000E10082FF0BC08091E20082FF07C080912B
:104C1000E1008B7F8093E1000E9464288091DA009C
:104C200080FF1FC08091D80080FF1BC08091DA00F8
:104C30008E7F8093DA008091D90080FF0DC080E1E3
:104C400089BD82E189BD09B400FEFDCF81E080937A
:104C5000EB020E94362205C019BC1092EB020E94A2
:104C600044228091E10080FF19C08091E20080FF22
:104C700015C08091E2008E7F8093E2008091E20077
:104C800080618093E2008091D80080628093D80098
:104C900019BC85E08093EB020E9449228091E100DB
:104CA00084FF30C08091E20084FF2CC080E189BD88
:104CB00082E189BD09B400FEFDCF8091D8008F7DCF
:104CC0008093D8008091E1008F7E8093E1008091F5
:104CD000E2008F7E8093E2008091E2008160809309
:104CE000E2008091E702882311F084E007C0809100
:104CF000E30087FD02C081E001C083E08093EB0206
:104D00000E9451228091E10083FF29C08091E2003E
:104D100083FF25C08091E100877F8093E10082E0DE
:104D20008093EB021092E7028091E1008E7F8093E6
:104D3000E1008091E2008E7F8093E2008091E200AA
:104D400080618093E20042E060E080E00E94EC2419
:104D50008091F00088608093F0000E944722FF91CC
:104D6000EF91BF91AF919F918F917F916F915F91E3
:104D70004F913F912F910F900FBE0F901F9018955C
:104D80001F920F920FB60F9211242F933F934F93C0
:104D90005F936F937F938F939F93AF93BF93CF93C3
:104DA000DF93EF93FF93C091E900CF708091EC0007
:104DB000D82FD17080FDD0E81092E9008091F000EA
:104DC000877F8093F00078940E9404271092E90076
:104DD0008091F00088608093F000CD2BCF70C0935D
:104DE000E900FF91EF91DF91CF91BF91AF919F913A
:104DF0008F917F916F915F914F913F912F910F9084
:104E00000FBE0F901F9018951F93CF93DF93CDB7D0
:104E1000DEB7AA970FB6F894DEBF0FBECDBFECEE9B
:104E2000F2E08091F100819322E0E43FF207C9F7BC
:104E30000E946F228091E80083FF2EC18091EC02D6
:104E40009091ED02492F50E04A30510508F024C1FD
:104E5000FA01EE59FF4F0C94D828803821F082389F
:104E600009F01AC108C08091E8029091E9029923E3
:104E700089F082600FC08091F0028F70873008F057
:104E80000BC18093E9008091EB0085FB882780F9B6
:104E90001092E9009091E800977F9093E80080934A
:104EA000F1001092F100D1C0282F2D7F09F0F4C03D
:104EB000882319F0823061F0EFC08091EE028130DA
:104EC00009F0EAC0933009F080E08093E9022EC037
:104ED0008091EE0281112AC08091F0028F702FEF35
:104EE000280F263008F0D8C08093E9002091EB000D
:104EF00020FF1CC0933021F48091EB00806214C02D
:104F00009091EB0090619093EB0021E030E0A901DB
:104F100002C0440F551F8A95E2F74093EA001092B1
:104F2000EA008091EB0088608093EB001092E9002A
:104F30008091E800877F8093E8000E942125ACC023
:104F40008111AAC01091EE021F778091E300807852
:104F5000812B8093E3008091E800877F8093E800B5
:104F60000E9421258091E80080FFFCCF8091E30022
:104F700080688093E300111102C082E001C083E0E9
:104F80008093EB0289C08058823008F085C0809100
:104F9000EE029091EF028C3D53E0950779F583E0A6
:104FA0008A838AE289834FB7F894DE01139620E062
:104FB0003EE051E2E32FF0E050935700E49120FFF0
:104FC00003C0E295EF703F5FEF708E2F90E0EA3004
:104FD00010F0C79601C0C0968D939D932F5F24312A
:104FE00049F74FBF8091E800877F8093E8006AE22D
:104FF00070E0CE0101960E942D2416C06091F0024F
:105000007091F102AE014F5F5F4F0E947123BC01AE
:10501000892B09F441C09091E800977F9093E800B4
:1050200089819A810E948B248091E8008B778093FC
:10503000E80032C0803881F58091E800877F809356
:10504000E8008091E7028093F1008091E8008E777C
:1050500072CF811121C08091EE029091EF029927C9
:105060000297D4F48091E800877F8093E8008091D4
:10507000EE028093E7020E9421258091E7028111D0
:1050800006C08091E30087FD02C081E001C084E09A
:105090008093EB020E945B228091E80083FF0AC0AC
:1050A0008091E800877F8093E8008091EB00806228
:1050B0008093EB00AA960FB6F894DEBF0FBECDBF6B
:1050C000DF91CF911F9108950895CF938091EB02C6
:1050D0008823A1F0C091E900CF709091EC00892F56
:1050E000817090FD80E8C82B1092E9008091E80063
:1050F00083FD0E940427CF70C093E900CF910895EB
:1051000087FB082E062687FD819567FD61950E9425
:105110000F290EF4919507FC81950895AA1BBB1BDE
:1051200051E107C0AA1FBB1FA617B70710F0A61BA7
:10513000B70B881F991F5A95A9F780959095BC01C8
:10514000CD01089597FB072E16F4009407D077FD44
:1051500009D00E948E2807FC05D03EF490958195D9
:105160009F4F0895709561957F4F0895A1E21A2E83
:10517000AA1BBB1BFD010DC0AA1FBB1FEE1FFF1FFB
:10518000A217B307E407F50720F0A21BB30BE40B4B
:10519000F50B661F771F881F991F1A9469F7609592
:1051A0007095809590959B01AC01BD01CF0108954C
:1051B000EE0FFF1F0590F491E02D09940E94E62860
:1051C000332312F48A1B9B0B0C94F728A29FB00187
:1051D000B39FC001A39F700D811D1124911DB29F2B
:1051E000700D811D1124911D08950E94E628B7FFBE
:1051F0000895821B930B08950E94E628A59F900DA9
:10520000B49F900DA49F800D911D11240895B7FFA8
:105210000C94FC280E94FC28821B930B0895991B78
:1052200079E004C0991F961708F0961B881F7A959D
:10523000C9F780950895FC014150504030F001902D
:105240000616D1F73197CF01089588279927089539
:10525000FB01DC0104C08D910190801921F44150C3
:105260005040C8F7881B990B0895F999FECF92BD5D
:1052700081BDF89A992780B50895A6E1B0E044E091
:1052800050E00C946F29A8E1B0E042E050E00C94AB
:105290006F29262FF999FECF92BD81BDF89A01970B
:1052A00000B4021639F01FBA20BD0FB6F894FA9A6E
:1052B000F99A0FBE08950396272F0E944A290E944B
:1052C0004929252F0E944A29242F0C944A29019606
:1052D000272F0E944A290C944929DC01CB01FC01AB
:1052E000F999FECF06C0F2BDE1BDF89A319600B43F
:0E52F0000D9241505040B8F70895F894FFCF4A
:1052FE00C8004302280850011E0A140101010200D1
:10530E000500050501191A1B1C1D1E1F2021229FB9
:10531E0021C221A32132222E22A22101E200E90084
:10532E00EA00B500B600B700CD008301CC008A01BB
:10533E009201940121022302240225022602270251
:10534E002A02B300B4006F007000818283E200E98C
:10535E0000EA00B500B600B700CD008301CC008A8C
:10536E000192019401210223022402250226022722
:10537E00022A02B300B4006F00700081828397C6C8
:10538E006636323331F7F6F591909294343500014A
:10539E00020202020606060909090909090F0F0F82
:1053AE000F0F0F151515181919191919191919198A
:0453BE00192324008B
:00000001FF
